:100000005A29A501A400B3172730A30010301420EB
:100010000330A300E8301420A30164301420A301AE
:100020000A30142024081F28A2002508A100240853
:10003000A00018212008031DB313B31B0800303E95
:1000400022280408A2008316051183120930A30098
:1000500003103120A20CA30B292803143120031410
:1000600055290318362800000511382805153828A9
:100070000030A1006230F228A60036088400093062
:10008000A70003104820A60CA70B422803144828F9
:100090008413B31D572800083404331D3406800030
:1000A000841700083404031C34068000622800080A
:1000B0003404031C340633193406800084173409D1
:1000C0008005622800308A00330D0639A0006F20B9
:1000D000A10000308A00200A6F200000F228733E41
:1000E00003188A0A82000134893403342934003425
:1000F00050340C34ED346400942003187B28AC2079
:10010000A801A2010930A300AD2094200318A80A79
:10011000AB1EA801A20CA30B8428AB1AA213A20D3C
:10012000AD20031422080800360884003408841720
:100130008004841300052B1B3406FF3E0800A40036
:100140002908031955295021A000240884002008FB
:100150008000A40AA903A02833172B081F39003EEA
:10016000A1002A08043E0318A10A331FF228331302
:10017000A0000310A10CA00C0310A10C200CF2286D
:10018000B31329080319B3170430A800250ECD2096
:100190002508CD20240ECD2024080F39F63E031863
:1001A000073E0A3ED328A000A8030319B313290869
:1001B0000319DD282802031808002008031DB313C3
:1001C000B31B0800303E5029A301A200FF30A20754
:1001D000031CA307031C55290330A100E330F220C0
:1001E000E628A101F43EA000A109FE30031CFB2873
:1001F000A0070318F828A0076400A10FF828000042
:1002000020180229201804290800A000A11B4A2157
:1002100020085529A2002008A6002408A0002608CE
:10022000A4002108A6002508A1002608A5001A2977
:10023000A501A4011030A600210DA40DA50D2208D2
:10024000A4022308031C230FA50203182E29220849
:10025000A40723080318230FA5070310A00DA10D61
:10026000A60B1C29200855291030A800A101A001C7
:10027000A70CA60C031C42292208A0072308031878
:10028000230FA107A10CA00CA50CA40CA80B3829C6
:1002900024085529A009A109A00A0319A10A0800E8
:1002A000840031088A00300882008313031383120C
:1002B0006400080088308B00831675308F0083122D
:1002C000073099008316133085009F0183129F0128
:1002D00083167F3081000330950083120930A3001C
:1002E000C430E520FE3022208030222042302220FF
:1002F000433022204D30222020302220473022203F
:100300006130222075302220673022206530222083
:10031000203022202030222056302220303022204F
:100320002E3022203030222031302220FE30222078
:10033000C0302220773022207730222077302220D0
:100340002E30222031302220353022203030222021
:100350006D30222070302220673022202E30222063
:10036000633022206F3022202E3022207530222050
:100370006B3022200730A300D030E520FE30222051
:10038000013022200530B6001030B4005430AA00ED
:100390002030AB007B20873C031DCA290B30A9000D
:1003A0007B30B000B10138309F200530B6001030EE
:1003B000B4005430AA002030AB007B20AA3C031DBF
:1003C000DD290B30A9007B30B000B10143309F2004
:1003D00064008518312A0730A300D030E520FE30B4
:1003E000222001302220FE302220803022200130C5
:1003F000D80064000930580203180E2A0230A90000
:100400005808383E84000008D2005208A400A50114
:100410002130B000B101C020D80FF929FE302220D0
:10042000C03022200130D80064000930580203187F
:10043000292A0230A9005808433E84000008D2004F
:100440005208A400A5012130B000B101C020D80F8E
:10045000142A0730A300D030E520FE3022200130DE
:1004600022203908A600A7010230A200A3013421EE
:10047000DA000F30BA053A08A600A7018030A200C2
:10048000A3013421D2002508D3003B085207D00035
:1004900053080318013ED100FE3022208030222074
:1004A0005A08012056302220203022205008A00077
:1004B0005108A1000A30A200A3011821D20021088E
:1004C000D3005308A500520802202E3022205008E5
:1004D000A0005108A1000A30A200A301182124089D
:1004E000D2002508D3005308A50052080220253069
:1004F0002220203022203C08A600A7018030A20044
:10050000A3013421D2002508D3003D08D2070318E7
:10051000D30A00305202CE000830031C013E5302C1
:10052000CF00CF1B5914CF1F59104F08A1004E0800
:100530000521CE002108CF004E08A6004F08A700D5
:10054000C430A2000930A3003421CE002508CF001A
:100550000230A30000300A21CE002108CF00640041
:10056000591CB52A2D302220B72A2B3022204E08C4
:10057000A0004F08A1006430A200A3011821CE0002
:100580002108CF004F08A5004E080220413022204C
:10059000203022202030222003103F0CD400D5012F
:1005A0000310400CD600D70164000518112B540825
:1005B000A6005508A7000930A200A3013421D200EB
:1005C0002508D3005208A0005308A1000530A2005E
:1005D000A3011821D2002108D30020305207D400F3
:1005E00053080318013ED5005608A6005708A70077
:1005F0000930A200A3013421D2002508D3005208FB
:10060000A0005308A1000530A200A3011821D200C8
:100610002108D30020305207D60053080318013EAA
:10062000D700FE302220C03022205508A5005408F3
:10063000022048302220203022205708A5005608EA
:1006400002204C302220203022204630222002304E
:10065000A9004808A400A5012130B000B101C020C4
:1006600020302220203022200530B6002030B40077
:100670000630B3005A083C200030591801303C20A5
:100680004E083C2050083C2054083C2056083C2092
:1006900048083C2064008518872B0530B6002030C0
:1006A000B4000630B30087303C20D80164000B3022
:1006B000580203186A2B0530B6002030B40006300B
:1006C000B3005808383E84000008D20052083C208D
:1006D000D80F562B0530B6002030B4000630B300DA
:1006E000AA303C20D80164000B3058020318872B35
:1006F0000530B6002030B4000630B3005808433E41
:1007000084000008D20052083C20D80F732BC22965
:02400E009C3CD8
:00000001FF
